:100000000C94E8010C942F020C942F020C942F02F4
:100010000C942F020C942F020C942F020C942F029C
:100020000C942F020C942F020C94751B0C94B11A93
:100030000C9448090C942F020C942F020C942F025C
:100040000C942F020C942F020C942F020C942F026C
:100050000C942F020C9407090C942F020C942F027D
:100060000C942F020C942F020C942F020C942F024C
:100070000C942F020C942F020C942F020C942F023C
:100080000C942F020C942F020C942F020C942F022C
:100090000C942F020C942F020C942F020C942F021C
:1000A0000C942F020C942F020C942F02C505C50549
:1000B000FF05FF05580674060A080A087F065D0753
:1000C0006E076E072C0B2C0B3F0B3F0B350B3F0BBA
:1000D0003F0B3F0B2C0B2C0B3A0B3F0B3F0B3A0B00
:1000E00021112411451152115A117A1112121212B2
:1000F0001212121212127D117F118411A911CB114B
:10010000CE11D111F311C518EC18931AEC18931AEB
:1001100038195B19931A501A601A00000000000089
:1001200000000000000000000000000000000000CF
:1001300000000000000000000000000000007E0F32
:1001400000D4FFFFFFC7000000780000000000009F
:1001500000002A2B28000000000000000000000022
:10016000000000000029000000002C1E3420212285
:1001700024342627252E362D3738271E1F202122EE
:10018000232425263333362E37381F040506070867
:10019000090A0B0C0D0E0F10111213141516171857
:1001A000191A1B1C1D2F3130232D35040506070895
:1001B000090A0B0C0D0E0F10111213141516171837
:1001C000191A1B1C1D2F3130354CA8004A00AE00F7
:1001D000015152004D00500051004F00005C0100E1
:1001E000780001000100C35CAC000100AB0001001D
:1001F00001000100010001000100010001000100F7
:1002000001000100010001000100010001000100E6
:10021000010005010902A10185020901A1000509EA
:1002200019012908150025019508750181020501AC
:10023000093009311581257F950275088106093835
:100240001581257F950175088106050C0A38021570
:1002500081257F950175088106C0C005010980A12F
:1002600001850319012AB700150126B7009501750C
:10027000108100C0050C0901A101850419012AA003
:1002800002150126A002950175108100C005010923
:1002900006A1018505050719E029E7150025019547
:1002A00008750181020507190029EF150025019540
:1002B000F07501810205081901290595057501915F
:1002C00002950175039101C00660FF0961A1010952
:1002D00062150026FF00952075088102096315004C
:1002E00026FF00952075089102C005010906A101AD
:1002F000050719E029E71500250195087501810218
:100300009501750881010507190029FF150026FFD1
:1003100000950675088100050819012905950575E0
:10032000019102950175039101C009025B0003016F
:1003300000A0FA09040000010301010009211101D4
:1003400000012240000705810308000A090401009A
:10035000020300000009211101000122220007050B
:1003600082032000010705030320000109040200A5
:10037000010300000009211101000122B600070558
:10038000840320000A120110010000000830349993
:100390009999990102000124035400680065002026
:1003A000006E00650069006E0020004B006500795A
:1003B0000062006F0061007200640000000C0364C2
:1003C00000690030006900620000000403090400B5
:1003D00011241FBECFEFDAE0DEBFCDBF04B603FEAF
:1003E00027C08091200290912102A0912202B09119
:1003F00023028730904BA740B04BD1F410922002DB
:1004000010922102109222021092230214BE84B78D
:10041000877F84BF0FB6F894A895809160008861AB
:1004200080936000109260000FBEE0E0F8E3099551
:1004300011E0A0E0B1E0E4E6FEE302C005900D9219
:10044000A435B107D9F722E0A4E5B1E001C01D92BF
:10045000A032B207E1F70E94530E0C94301F0C94A7
:1004600000003F924F925F926F927F928F929F9285
:10047000AF92BF92CF92DF92EF92FF920F931F93B2
:10048000CF93DF93CDB7DEB729970FB6F894DEBFD1
:100490000FBECDBFFC018081918123813481232B4C
:1004A00031F09F3F31F491E08F3F19F403C091E0A8
:1004B00001C090E090FDEBC57F0185E0DE01119663
:1004C00001900D928A95E1F7F701228189819A8145
:1004D000222349F00E94CD0A182F682F89819A8122
:1004E0000E946F0B03C00E94430B182F69817A8111
:1004F000812F0E9473148C01F7018281882309F4F3
:10050000F1C0980122513F452031310508F018C152
:100510008FEF93E00E94B91E8111EEC002513FE6B9
:10052000832E912C002379F08114F4E09F0609F4C6
:10053000E3C0C4010E94B91E811101C001501FEF28
:10054000811A910AEFCF1E821F82188619864424D1
:1005500043942AE0322E84010F5F1F4FC4010E9492
:10056000B91E8E831F82882309F4C6C09FEF980F9F
:10057000933060F48F834E8222E0820E911CC8017A
:100580000E94B91E8887811102C0B6C048018E0141
:100590000A5F1F4FF80120812223E9F2213009F080
:1005A0004CC08181813049F46801F2E0CF0ED11C4A
:1005B000F80182810E94E91D0AC0823051F468016D
:1005C000F2E0CF0ED11CF80182810E94251D860128
:1005D00086C0833049F46801F2E0CF0ED11CF801E7
:1005E00082810E94BE1CF3CF843019F00F5F1F4F31
:1005F00076C0F80122810E5F1F4F80E090E030E06E
:10060000205331092A30310568F4389EA001399E03
:10061000500D1124C901840F951F0F5F1F4FF80162
:100620002081EDCF009709F45AC0EFE9FFE0319740
:10063000F1F700C000000197F5CFE22FF0E0E65B94
:10064000FE4F5490822F86958695869590E0FC010A
:10065000E65CFE4F64902770712C022E02C07594E8
:1006600067940A94E2F7F1E06F227724FC01E65DDB
:10067000FE4FA490B12C022E02C0B594A7940A9408
:10068000E2F731E0A322BB24FC01E65EFE4FC490FA
:10069000D12C02C0D594C7942A95E2F781E0C822F4
:1006A000DD246114710419F081EE0E94251DA1144E
:1006B000B10419F086EE0E94251D852D0E94E91DCA
:1006C000AB2819F086EE0E94BE1C672819F081EE57
:1006D0000E94BE1CCD2819F08CE20E94E91D0F5F1C
:1006E0001F4F58CF00313FE5130709F0C7C481E021
:1006F0000E94A40B0E94C1178091BB01877009F46E
:10070000C6C4F7018281882309F4C1C482E0299616
:100710000FB6F894DEBF0FBECDBFDF91CF911F9112
:100720000F91FF90EF90DF90CF90BF90AF909F9090
:100730008F907F906F905F904F903F900C94C90B7B
:100740000031FFE51F0711F481E005C001312FE5FD
:10075000120721F482E00E94E60BCCCF033FFCE5B8
:100760001F0799F406E221EE40EE63EF7CE509C035
:10077000073DECE51E0711F506E221EE41EE67EDBF
:100780007CE5C7010E949613B7CF043F2CE5120702
:1007900008F03FC1083D3CE5130731F407E225EEC0
:1007A00045EE68ED7CE5EDCF093D9CE5190701F7C5
:1007B00008E221E045EE69ED7CE5E3CF882309F40A
:1007C0005DC11092560102309CE5190708F440C142
:1007D0000631ECE51E0730F0C8018A5F9C45099799
:1007E00008F036C10E94CE099093C5018093C401E0
:1007F0000031FCE51F0709F4C3C008F041C0083010
:100800003CE5130709F49AC0F0F404309CE519079D
:1008100009F487C068F40230FCE51F0709F477C0CB
:1008200003301C4509F0E5C08091C401826076C0A8
:1008300006303CE5130709F46EC008F07BC08091D8
:10084000C40188606BC00C309CE5190709F485C0B1
:1008500068F40A30FCE51F0709F474C008F079C099
:100860000E94360E8091C401806858C00E303CE56D
:10087000130709F476C008F07FC08091C4018BC0D3
:100880000B3F9CE5190709F44FC018F50331FCE54F
:100890001F0709F47DC078F401313CE5130709F422
:1008A00073C002311C4509F0A4C00E94360E80912D
:1008B000C4018F7733C005319CE5190709F472C074
:1008C00008F486C00A3F1C4509F093C08091C50119
:1008D0003EC00F3F2CE5120709F45FC058F40D3FEE
:1008E0008CE5180709F444C008F43FC08091C501A5
:1008F00082602DC00130EDE51E0709F475C008F4D3
:100900005DC002301D4509F074C060E06EC080918A
:10091000C401816003C08091C40180618093C401DF
:1009200068C08091C40111C08091C501826080932C
:10093000C5015FC08091C4018062F0CF8091C40185
:100940008064ECCF8091C40188608460E7CF8160CF
:10095000EECF8091C4018E7FE1CF8091C4018D7F65
:10096000DDCF8091C401877FD9CF8091C50118C0A8
:100970008091C5018D7FDBCF8091C4018F7ECECF6A
:100980008091C4018F7DCACF8091C4018F7BC6CF77
:100990008091C401877F8B7FC1CF8091C5018D7FFE
:1009A0008E7FC5CF8091C40182FB222720F991E080
:1009B000922790FB82F990FB83F9B0CF8091C5011B
:1009C000982F909591708E7F892B90FB81F9AFCFF6
:1009D0000E94360E8091C40187FB222720F991E006
:1009E000922790FB87F99ACF61E08EE090E00E9419
:1009F000C71E6091C4011091C50184E090E00E947F
:100A0000C71E612F82E290E00E94C71E0E94360E30
:100A100073CE053FFCE51F0731F406E221EE42EEFE
:100A200065EF7CE5AECE053F2CE5120730F407E21A
:100A300025EE44EE64EF7CE5A4CE063F3CE51307CB
:100A400009F0BCCE07E225EE46EE66EF7CE599CED6
:100A500006318CE5180711F58091BE018A7A91E084
:100A600009F490E090935701882311F065E301C0E9
:100A700069E288E591E00E9499090DC006311C45A4
:100A8000F1F580915701882309F4FFC265E388E5F9
:100A900091E00E9471090E94500A2ECE0A353DE570
:100AA000130741F150F401159CE51907A9F00E3D1B
:100AB0001C4529F50E94DF091FCE0B35FDE51F07F8
:100AC000D9F00C351D45D9F48091C50182FB8827EA
:100AD00080F991E0892711C00E94360E3FEF84E330
:100AE0009CE0315080409040E1F700C000000E943F
:100AF000F60802CE81E001C080E00E94B30AF7014F
:100B0000828100811181882349F0C8010E94CD0AA9
:100B1000D82E682FC8010E946F0B04C0C8010E9424
:100B2000430BD82EB8018D2D0E9432168C01982EC1
:100B3000F701D280A580A2949FE0A9228091BB01F9
:100B4000877099F0DD2089F0812F807F803421F03B
:100B500080E2800F883048F082E00E94C90B8091CB
:100B6000BB018770CC24C3948111C12CB12EB294E7
:100B70008FE0B8228B2D90E08C30910508F04AC2AE
:100B8000FC01EA5AFF4F0C940F1F812F807F1F70CA
:100B9000882311F01295107FDD20B9F0112309F49C
:100BA00024C280E2800F883010F0911006C080913E
:100BB000BE01182B1093BE0105C08091BD01182BFA
:100BC0001093BD010E94500A10C2802F0E94BE1CCB
:100BD000112309F41FC2005E1095083010F0911027
:100BE00006C08091BE0118231093BE0105C08091FC
:100BF000BD0118231093BD010E94500A0BC2812F22
:100C0000807F1F70803211F01295107F992021F0A3
:100C1000F1E09F1611F130C0DD20B1F0AA2081F083
:100C200001E0A0120DC08091C50182FDF3C1809149
:100C3000BF01182B181709F4EDC11093BF01EAC1C9
:100C40008091BF01812B10C0AA2021F021E0A216C3
:100C500009F4E0C10E944A0A27C0DD2041F035E0D6
:100C60003A1508F4D7C1812F0E94B41CD3C184E087
:100C70008A1508F4CFC118C0DD2049F0AA2099F3E5
:100C8000F701858180FFB1C18F708583ECCFAA20E9
:100C900059F0093309F0BBC1FFEF17EE23E0F15023
:100CA00010402040E1F7B1C1812F0E94A91CB2C1C0
:100CB000812F86958695837019F0813059F0AAC1ED
:100CC000DD2019F0C801937002C080E090E00E941E
:100CD0007413A6C1DD2019F0C801937002C080E032
:100CE00090E00E945E139CC1802FDD2019F00E94CD
:100CF000631502C00E94AA140E94801491C1812F22
:100D0000837009F069C0D11089C1902F9295969592
:100D10009770990F990F802F8F70882E912CA12C8E
:100D2000B12C092E04C0880C991CAA1CBB1C0A9467
:100D3000D2F704FF12C04FE050E060E070E004C062
:100D4000440F551F661F771F9A95D2F7DB01CA0122
:100D500080959095A095B09503C080E090E0DC016F
:100D600016951695412F4370423019F1C8F4009141
:100D7000C0011091C1012091C2013091C3014130E5
:100D800059F088299929AA29BB29BC01CD016023E2
:100D90007123822393230AC0802A912AA22AB32A8C
:100DA000BC01CD01682979298A299B290E94070C59
:100DB00035C188299929AA29BB290091C001109120
:100DC000C1012091C2013091C301BC01CD01602756
:100DD000712782279327EACFDD2019F0812F8170B8
:100DE00001C08695882309F419C1902F9295969594
:100DF0009770990F990F802F8F70882E912CA12CAE
:100E0000B12C092E04C0880C991CAA1CBB1C0A9486
:100E1000D2F704FF12C04FE050E060E070E004C081
:100E2000440F551F661F771F9A95D2F7DB01CA0141
:100E300080959095A095B09503C080E090E0DC018E
:100E400016951695412F43704230D9F068F5009100
:100E50001C0210911D0220911E0230911F02413090
:100E600059F088299929AA29BB29BC01CD01602301
:100E70007123822393231EC0802A912AA22AB32A97
:100E800013C088299929AA29BB2900911C02109115
:100E90001D0220911E0230911F02BC01CD0160276E
:100EA00071278227932706C0BC01CD0168297929C3
:100EB0008A299B290E949A0BB1C01F70DD2039F04E
:100EC000812F0E94E60B802F0E94B41CA7C0802FA8
:100ED0000E94A91C812F0E94A40BA0C0802F32EF7A
:100EE000931609F440C0391538F090EF991661F067
:100EF000E1EF9E1699F174C0F3EF9F16D9F124EF3C
:100F0000921609F44EC06CC0DD2019F134E03A1598
:100F100008F480C01F7181E090E0A0E0B0E0AC0177
:100F2000BD0104C0440F551F661F771F1A95D2F7E5
:100F300080911C0290911D02A0911E02B0911F028F
:100F40008A019B01082719272A273B27C901B801D5
:100F500025C025E02A1508F45DC0DCCFDD2029F08E
:100F6000812F8F7130C0DD20D9F3812F8F710E94C6
:100F7000A40B50C0DD2079F01F7181E090E0A0E06B
:100F8000B0E0BC01CD0104C0660F771F881F991F18
:100F90001A95D2F703C060E070E0CB010E949A0B73
:100FA00039C0DD2099F01F71812F0E94E60B8091DE
:100FB000C50182FD07C038E0139FC0011124836082
:100FC0008093BB01812F0E94E60B24C081E00E9428
:100FD000C90B81E08A15F0F482E00E94C90B1AC0A7
:100FE000DD2039F0AA2009F4BBCF802F0E94251DF7
:100FF00011C0AA2009F4B9CF893349F49FEFE7EE75
:10100000F3E09150E040F040E1F700C00000802F95
:101010000E94BE1C88EF8B0D843010F40E948A134E
:10102000CC20A9F18091BB0180FD31C0F701128273
:101030008595859585950E94E60BC7010E94310232
:101040008091BB0185958595859529960FB6F89475
:10105000DEBF0FBECDBFDF91CF911F910F91FF90EB
:10106000EF90DF90CF90BF90AF909F908F907F9048
:101070006F905F904F903F900C94A40B01319FE5CF
:10108000190709F06BCB82E033CB69E200CD2996DA
:101090000FB6F894DEBF0FBECDBFDF91CF911F9189
:1010A0000F91FF90EF90DF90CF90BF90AF909F9007
:1010B0008F907F906F905F904F903F9008958091B8
:1010C000EF01089580E0089524E02093E9002FEFD8
:1010D0003091E800215035FD06C035ED3A95F1F725
:1010E00000002111F5CF2091E80025FF0BC040E062
:1010F00050E066E070E00E947D1C8091E8008E77F1
:101100008093E8000895CF93DF9320910A01222372
:1011100039F02091C40127FF03C060E224E002C03F
:1011200068E021E02093E9002FEF3091E8002150A2
:1011300035FD06C035ED3A95F1F700002111F5CFE8
:101140002091E80025FF1DC0EC0180910A0181116A
:1011500005C040E050E068E070E003C070E040E0AF
:1011600050E0CE010E947D1C8091E8008E77809334
:10117000E80080E2FE01A0EFB1E001900D928A95B7
:10118000E1F7DF91CF910895CF93DF9300D01F92C5
:10119000CDB7DEB790911202943011F589837B832D
:1011A0006A839093E9008FEF9091E800815095FD5C
:1011B00006C095ED9A95F1F700008111F5CF809169
:1011C000E80085FF0DC040E050E063E070E0CE0134
:1011D00001960E947D1C8091E8008E778093E80044
:1011E0000F900F900F90DF91CF91089587E797E7C9
:1011F00090930108809300089AE088E10FB6F89474
:10120000A895809360000FBE90936000FFCF789404
:101210001F920F920FB60F9211248F939F93AF934B
:10122000BF938091E0019091E101A091E201B09122
:10123000E3010196A11DB11D8093E0019093E101AE
:10124000A093E201B093E301BF91AF919F918F9181
:101250000F900FBE0F901F9018959C014FB7F894F8
:101260008091E0019091E101A091E201B091E30150
:101270004FBF821B930B08952FB7F8948091E00124
:101280009091E101A091E201B091E3012FBF089597
:101290001F920F920FB60F9211248F939F93AF93CB
:1012A000BF938091CB01811113C08091E001909197
:1012B000E101A091E201B091E3014196A11DB11DB0
:1012C0008093E0019093E101A093E201B093E301E8
:1012D000BF91AF919F918F910F900FBE0F901F9074
:1012E000189520910A012223C9F02091C40127FFFB
:1012F00015C0262F2695269526952E31C8F4FC017B
:10130000E20FF11D677081E090E001C0880F6A95DF
:10131000EAF780959281892382830895FC010696DD
:101320002281621301C012823196E817F907C1F7D2
:10133000089520910A012223C1F02091C40127FFC2
:1013400014C0262F2695269526952E3130F5FC01C2
:10135000E20FF11D677081E090E001C0880F6A958F
:10136000EAF79281892B82830895FC0132962FEF50
:1013700030E04191641789F02F3F19F4411101C009
:10138000232F3F5F3630A9F72F3F39F0FC01E20FE2
:10139000F11D27FDFA95628308950895CF9384E0A7
:1013A00090E00E94B91EC82F82E290E00E94B91E10
:1013B0002C2F30E0A901582BCA01CF9108956AEE75
:1013C0007EEF80E090E00E94E51E60E082E090E029
:1013D0000E94C71E60E083E090E00E94C71E10924A
:1013E000C0011092C1011092C2011092C30160E0CD
:1013F00084E090E00E94C71E60E082E290E00E94DC
:10140000C71E60E085E090E00E94C71E60E086E0B5
:1014100090E00E94C71E6FEF87E090E00E94C71E19
:1014200040E050E0BA0188E090E00E94D91E60E000
:101430008DE090E00E94C71E40E050E0BA0188E1D4
:1014400090E00E94D91E60E087E190E00E94C71EF4
:1014500040E050E0BA018CE190E00E94D91E60E0CB
:1014600070E080E290E00E94E51E40E050E0BA01AA
:1014700088E190E00E94D91E40E050E0BA018FE080
:1014800090E00E94D91E40E050E0BA0183E190E074
:101490000C94D91E8091BF0181111092BF01089553
:1014A0009091BE018091BD01892B2091BC01982FA4
:1014B000922B909358018091BF018823D9F0892BFA
:1014C0008093580180910A01882331F08091C401F2
:1014D00087FF02C08EE101C086E0EAE5F1E090E01E
:1014E000815028F021912223D9F39F5FF9CF9111E8
:1014F0000E944A0AE091C901F091CA013097A9F00F
:1015000080910A01882359F08091C40187FF07C0A8
:10151000809158018093590185E0809358010280A1
:10152000F381E02D88E591E00994089580E090E052
:101530000E94741380E090E00E945E131092BD013F
:101540001092BC010E94500AE2EDF1E086E0DF015A
:101550001D928A95E9F71092CF011092CC0110925A
:1015600078010C948014CF93C091C501C2FB9927D8
:1015700090F9981781F080FBC2F9C093C501609182
:10158000C40184E090E00E94C71E6C2F82E290E0CC
:10159000CF910C94C71ECF910895BF92CF92DF9246
:1015A000EF92FF920F931F93CF93DF938C01C09024
:1015B0001C02D0901D02E0901E02F0901F0280914C
:1015C000C0019091C101A091C201B091C301C82A8C
:1015D000D92AEA2AFB2ACFE1D0E0D701C6010C2E96
:1015E00004C0B695A795979587950A94D2F780FD84
:1015F00004C0219790F7B12C07C0BC2EB8018C2FE6
:101600000E9432160197A9F38B2DDF91CF911F9184
:101610000F91FF90EF90DF90CF90BF900895CF9300
:10162000DF93EC010E94CD0ABE010E943216DF91C9
:10163000CF9108950E940F0B292F2F70E92FE2956B
:10164000EF704E2F50E0FA013297EE30F105B8F40A
:10165000EE59FF4F0C940F1F803F99F018F4883E0D
:1016600070F40FC0843F59F40CC0883E50F0813FA5
:1016700031F407C0822F869586958695089580E07F
:10168000089581E00895292F220F920F890F682F66
:10169000669566956695982F977085E0689FB0016E
:1016A000112440E050E080E0FB01E40FF51FEF540F
:1016B000FE4F208130E0092E02C0369527950A940E
:1016C000E2F721703327042E01C0220F0A94EAF7B3
:1016D000822B4F5F5F4F4530510531F70895292F19
:1016E000220F920F890FE82FE695E695E695877011
:1016F00051E001C0550F8A95EAF785E0E89FF001B7
:101700001124EF54FE4F20E030E070E04081CB0127
:10171000022E02C0969587950A94E2F78170819512
:1017200084278523842781932F5F3F4F2530310500
:1017300069F7089560931C0270931D0280931E0246
:1017400090931F020C94960A0F931F9341E050E070
:1017500060E070E004C0440F551F661F771F8A9534
:10176000D2F7409550956095709580911C029091AC
:101770001D02A0911E02B0911F028A019B01082345
:1017800019232A233B23C901B8011F910F910C94FF
:101790009A0B2091BB01809582238093BB01982FE7
:1017A000977041F430E0482F082E000C550B241799
:1017B000350721F49091C50192FF07C08595859565
:1017C00085950E94A40B1092BB0108950F931F935F
:1017D00041E050E060E070E004C0440F551F661F18
:1017E000771F8A95D2F780911C0290911D02A091DB
:1017F0001E02B0911F028A019B01082B192B2A2B74
:101800003B2BC901B8011F910F910C949A0B609367
:10181000C0017093C1018093C2019093C3010C94E5
:10182000960A8091B00190917F01891719F08F5F1E
:101830008770FBCF08950F931F93CF93DF93809111
:101840007E0182958F7009F05DC080917B018823B5
:1018500009F458C08091B00110917F016091790125
:1018600070917A01C0917C01D0917D0191E06F3F30
:1018700009F090E0292F06E0811709F443C0209772
:1018800021F07F3F21F030E003C031E001C0322F72
:1018900090E030FD34C0089FF001099FF00D112445
:1018A000DF01A058BE4F11963C911197371327C006
:1018B0003C91361324C012963C91129731111FC0EF
:1018C00013964D915C9114974C1B5D0B483C510550
:1018D000B0F480917E018F70806180937E01EB5720
:1018E000FE4F80818F708061808389E791E00E9444
:1018F0003102DF91CF911F910F910C94110C019641
:101900008770BACFDF91CF911F910F9108959F9269
:10191000AF92BF92CF92DF92EF92FF920F931F93FD
:10192000CF93DF93CDB7DEB761970FB6F894DEBFE4
:101930000FBECDBF8C0185E0F801DE011D96019040
:101940000D928A95E1F7F80190818181E2803091D2
:10195000790160917A0140917C0150917D0141159E
:10196000510531F06F3F31F421E03F3F19F403C0DE
:1019700021E001C020E0F22FF1709F2E20FD23C155
:10198000F801C380D48029E7A22E21E0B22EF09086
:101990007B01F601E41BF50BFF2009F4CEC020917A
:1019A0007E01E83CF10508F099C0422F407F09F024
:1019B00051C0681311C039130FC0FE2CE1100CC0C8
:1019C0002F70206120937E01C5010E943102809119
:1019D0007E01F801858337C1CD2831F08F3F31F486
:1019E00021E09F3F19F403C021E001C020E020FD69
:1019F00003C021E02E2502C020E030E0F22FF1707C
:101A0000FF2E20FF1DC02091B00140917F0156E0C4
:101A1000241709F4F6C030E0529FF001539FF00DF7
:101A20001124E058FE4F6181861306C06081961331
:101A300003C06281E61204C02F5F3F4F2770E8CFDA
:101A4000FE2CEE2009F4FFC080917E01816080931E
:101A50007E0150C0681307C0391305C0E11003C0F0
:101A6000F80125838DC09D878E878D859E850E9478
:101A70001A0B882369F1EE2059F120917E01822F03
:101A800082958F7090E0029774F080917901909127
:101A90007A0198878F831986DB86CA862C87CE01C8
:101AA00007960E94310286E0F801A9E7B1E00190B3
:101AB0000D928A95E1F70E941B0C0DC06817E1F0AA
:101AC0009D878E878D859E850E941A0B81111EC071
:101AD000C8010E943102FF24F394B5C0422F407F19
:101AE00069F789E791E00E94310286E0F5011192E1
:101AF0008A95E9F7F12CA7C03913E2CFE110E0CFC6
:101B0000F8012583C8010E94310257C0EE2001F37D
:101B100020917E01822F82958F7090E002971CF2B7
:101B20008091790190917A019A8389831B82DD8269
:101B3000CC822E83CE010196B4CFE83CF105E8F5C6
:101B4000FE2CEE2029F2681327C0391325C02091FE
:101B50007E0120FD18C0822F82958F70482F50E0A3
:101B60004115510581F0F80125834F30510541F0B1
:101B70008F5F982F9295907F822F8F70892B85830E
:101B8000C8010E94310286E0F801A9E7B1E00190A6
:101B90000D928A95E1F757C09D878E878D859E852A
:101BA0000E941A0B81117FCF80917E01816080930A
:101BB0007E01C8010E94310246C086E0F501119203
:101BC0008A95E9F740C0EE2009F482CF9D878E8781
:101BD0008D859E850E941A0BF82E882309F478CFF4
:101BE00086E0F801A9E7B1E001900D928A95E1F74E
:101BF0008091790190917A010E940F0B0E941B0C39
:101C000022C09D878E878D859E850E940F0B292F70
:101C100022952F70223028F49F7039F0811105C071
:101C20000BC0243028F49F7049F4805E883020F087
:101C3000C8010E9431029F2CF92C05C0F801958142
:101C4000907F99F7F9CF8F2D61960FB6F894DEBF8C
:101C50000FBECDBFDF91CF911F910F91FF90EF90FD
:101C6000DF90CF90BF90AF909F9008951092BE01EB
:101C700080910A01882331F08091C40187FF02C05E
:101C80008EE101C086E0EAE5F1E0DF011D928A9570
:101C9000E9F70C94960ABC0184E00C94C408BC01DA
:101CA00083E00C94C408CF93DF93CDB7DEB7AA9737
:101CB0000FB6F894DEBF0FBECDBF84B7877F84BF59
:101CC0000FB6F894A89580916000886180936000B9
:101CD000109260000FBE90E080E80FB6F8948093F9
:101CE0006100909361000FBE85B7806885BF85B79E
:101CF000806885BF82E698E09093550180935401F7
:101D00000E94F51A0E94141B8091E2008460809367
:101D1000E2007894809112028823A1F01091E900EA
:101D20001F709091EC00892F817090FD80E8182B36
:101D30001092E9008091E80083FD0E94DF171F7078
:101D40001093E90082E084BD93E095BD9AEF97BDC2
:101D500080936E004BE051E0A4E1B1E001E010E0BF
:101D600020E030E0FA01E20FF31F80818F3FA1F005
:101D7000E82FE295EF70F0E061A18F70780102C06A
:101D8000EE0CFF1C8A95E2F7C7019E2D90959623D5
:101D900091A392A1892B82A32F5F3F4F233031055E
:101DA00009F74D5F5F4FA417B507D1F61092C60132
:101DB0001092DD011092C7011092DE011092C8014D
:101DC0001092DF0180E090E00E94C11E8A3E9E4F8B
:101DD00011F00E94DF0982E090E00E94B91E80931A
:101DE000D9010E94CE099093C5018093C4010E943D
:101DF000BE158FE39CE90197F1F700C000000E9437
:101E0000BE158091DD0180FF17C06FEF83E290E087
:101E10000E94C71E6FEF84E290E00E94C71E6FEF22
:101E200085E290E00E94C71E6FEF7FEF80E090E0B8
:101E30000E94E51E0E94F60883E090E00E94B91E11
:101E4000682F70E080E090E00E94070C83E290E051
:101E50000E94B91E813281F484E290E00E94B91E92
:101E6000873051F485E290E00E94B91E91E0833101
:101E700009F090E0892F01C080E080FF1BC380E063
:101E800091E09093CA018093C90198E1C92ED12CA9
:101E900020E4422E30E1532E42E1842E50E1952E73
:101EA0008E010F5F1F4F80911202853009F042C0F2
:101EB00080911202853009F039C08091120284307D
:101EC00009F11092CB010FB6F894A895C09260006A
:101ED0000FBE4092600083B7817F846083BF83B769
:101EE000816083BF7894889583B78E7F83BF0FB658
:101EF000F894A895809160008861809360001092AA
:101F000060000FBE80911102882391F20E94BE15DD
:101F10008091DD018111B0C28091DE018111ACC2DE
:101F20008091DF01882309F4C3CFA6C20E94360E38
:101F30000E948A130E94BE15882359F08FB7F89427
:101F40004091E0015091E1016091E2017091E30163
:101F50008FBFEDEDF1E0AAEDB1E0E12CF12C3E2DCB
:101F600021919D91922721F180E0BB24B394492FC8
:101F70004B21D1F089A33AA32B2181E009F480E021
:101F80008BA30E943C098160782F9DA38CA349A15B
:101F90005AA16BA18DA10E94C012F701E652FE4F1B
:101FA0008081B826B0821BC08F5FBB0C8330F9F6EE
:101FB0009FEFE91AF90A23E0E216F10481F68FEFA8
:101FC0008EA38FA318A60E943C098160782F9AA740
:101FD00089A74EA15FA168A58AA50E94C01286E0CC
:101FE000E2EDF1E0D80101900D928A95E1F7A09021
:101FF000D401B090D501E090D601F090D7011092B5
:10200000D4011092D5011092D6011092D701A110DF
:1020100003C0BB2009F451C08091D0019091D1013F
:102020000E942D099C019091CF01992309F45BC274
:102030002333310508F441C09F3F19F09F5F90930F
:10204000CF01AA2061F00E9443151A1414F491E004
:1020500001C09FEF899F802D11248093D401BB2064
:1020600061F00E9443151B1414F491E001C09FEF2E
:10207000899F802D11248093D5013091D401332381
:10208000E1F02091D5012223C1F045EB3403C001DA
:102090001124992319F09093D40103C081E0809317
:1020A000D40135EB2303C0011124992319F0909337
:1020B000D50103C081E08093D501E11003C0FF206A
:1020C00009F451C08091CD019091CE010E942D095B
:1020D0009C019091CC01992309F40AC2253631055F
:1020E00008F441C09F3F19F09F5F9093CC01EE2010
:1020F00061F00E9421151E1414F491E001C09FEFBD
:10210000899F802D11248093D601FF2061F00E94C9
:1021100021151F1414F491E001C09FEF899F802DB9
:1021200011248093D7013091D6013323E1F020911F
:10213000D7012223C1F045EB3403C00111249923B8
:1021400019F09093D60103C081E08093D60135EB5E
:102150002303C0011124992319F09093D70103C0E0
:1021600081E08093D7018091D40181110BC08091CF
:10217000D501811107C08091D601811103C08091E2
:10218000D70181110E948014AB82BC82ED82FE8255
:1021900086E0F801A2EDB1E001900D928A95E1F799
:1021A0000E948A139091D801891721F00E948A1306
:1021B0008093D80180911202843009F074CE83E0BC
:1021C0008093E9008091E80082FF6DCE8091E80065
:1021D00085FF21C00E944A1C81111BC080E2E82EAD
:1021E000F12C580109C08091F100F50181935F0144
:1021F000F1E0EF1AF10869F08091E80085FDF3CF76
:102200008091E8008B778093E8000E944A1C882325
:1022100099F391E001C090E08091E8008B77809382
:10222000E800992309F43FCEE9818E2F90E0FC016C
:102230003197E331F10508F0F5C0E059FF4F0C94F8
:102240000F1F1A8289E05EC08A81823009F42AC198
:10225000833089F0813009F0E5C02FB7F894809180
:10226000E0019091E101A091E201B091E3012FBF63
:10227000BB83AC831CC08091DD018B838091DE0128
:102280008C838091DF018D83CFC08A81823009F0F9
:10229000C9C06B817C818D819E810E94151F86E261
:1022A00090E025C04C816B818A810E944D149D83F2
:1022B0008E83BAC0AD80BE80BA24AB24BA248C8190
:1022C000EB809A8126E0E29E7001112432E1939F17
:1022D000E00CF11C1124E80EF11CE80EF11C6B2D32
:1022E000C70187960E94C71E6A2DC70188960E9463
:1022F000C71E9AC00E94191497C09A8295C083E0A5
:102300008A8381E98B8390C0EA80FB80FE24EF24DE
:10231000FE24AC80B12C3801C70181599F4F930135
:10232000201B310B2A153B0508F07EC041E9E4165D
:1023300043E0F40628F40E94B91EF301848302C02E
:10234000F3011482FFEFEF1AFF0A2FEF621A720AED
:10235000E3CFEA80FB80FE24EF24FE24AC80B12C86
:102360003801C70181599F4F9301201B310B2A155A
:102370003B0508F059C031E9E31633E0F30620F4D9
:10238000F30164810E94C71EFFEFEF1AFF0A2FEFCF
:10239000621A720AE6CF0E94091446C084E08A835A
:1023A00043C0EA80FB80FE24EF24FE24AC80B12CE5
:1023B0003801C70187969301201B310B2A153B0575
:1023C00098F538E4E316F10428F40E94B91EF301ED
:1023D000848302C0F3011482FFEFEF1AFF0A2FEF8C
:1023E000621A720AE6CFEA80FB80FE24EF24FE2404
:1023F000AC80B12C3801C70187969301201B310BAB
:102400002A153B0588F438E4E316F10420F4F301BF
:1024100064810E94C71EFFEFEF1AFF0A2FEF621AB6
:10242000720AE9CF8FEF898380911202843009F01C
:102430003ACD8091E9008F702091EC00922F91703D
:1024400020FD90E8F92EF82A82E08093E90080913F
:10245000E80080FF0CC040E050E060E270E0C8019E
:102460000E947D1C8091E8008E778093E8008F2D7C
:102470008F708093E90017CD59BC89BC09B400FE68
:10248000FDCF8091D8008F7D8093D8008091E000AF
:1024900082608093E0008091E00081FDFCCF0E948B
:1024A000360E06CD86E290E00E94B91E1B821C8289
:1024B0001D82FECE60E086E290E00E94C71E0E9470
:1024C00019140E94091461E283E290E00E94C71E81
:1024D00067E084E290E00E94C71E63E185E290E03D
:1024E0000E94C71ECCCC2D32314008F0A7CDE5CDDF
:1024F0002D32314008F0F8CD36CE9091C40192FFD4
:102500000DC0282F2871283019F4877F846006C0F9
:10251000282F2471243011F48B7F886093FF0DC025
:10252000282F2871283119F4877E846106C0282F4E
:102530002471243111F48B7E88612091C50120FF24
:102540000DC0382F3871383019F4877F816006C08C
:10255000382F3171313011F48E7F886021FF0DC02A
:10256000282F2871283119F4877E816106C0282F11
:102570002171213111F48E7E886194FD877E08954A
:102580001F93CF93DF93CDB7DEB767970FB6F8945D
:10259000DEBF0FBECDBF342F4B8B252F5C8B6D8BD9
:1025A0007E8B8F8B4E895F8961111092BD0186E011
:1025B000FE013D96DF01982F1D929A95E9F73D8720
:1025C0002E876F87598B488BDE01179601900D92ED
:1025D0008A95E1F7CE0107960E94870C81113EC0D3
:1025E00086E0FE013796DE01119601900D928A95E4
:1025F000E1F7FF81E8856A857B856115710531F01A
:10260000EF3F31F481E0FF3F19F403C081E001C0E6
:1026100080E080FD23C020917F0130E0C901019658
:10262000877099274091B00150E08417950779F1A0
:10263000F983EA837D836C8396E0929FD001939F18
:10264000B00D1124A058BE4FFE01319601900D929D
:102650009A95E1F780937F010E94110C16E080911A
:10266000B00190917F018917F9F0189FC0011124E2
:1026700080589E4F0E94870C8823B1F08091B00152
:1026800090E00196877099278093B001E8CF0E946F
:10269000360E10927F011092B001E9E7F1E086E07A
:1026A000DF011D928A95E9F767960FB6F894DEBFB1
:1026B0000FBECDBFDF91CF911F9108952091EB0107
:1026C0003091EC012817390771F09093EC01809359
:1026D000EB01E091C901F091CA01309721F000842B
:1026E000F185E02D099408952091E9013091EA01E6
:1026F0002817390771F09093EA018093E901E0917E
:10270000C901F091CA01309721F00680F781E02DD0
:1027100009940895E091C901F091CA01309721F020
:102720000190F081E02D099480E008950F931F93AC
:10273000CF93DF93C42FD22FFC0182818823C9F06D
:10274000409356010E943C099093E8018093E70171
:1027500080E28C0F883008F057C0C77081E001C05C
:10276000880FCA95EAF7DF91CF911F910F910C94D2
:10277000B41C80915601481330C08091E7019091BC
:10278000E8010E942D09883C910538F510E21D0FE3
:10279000CD17B9F080E28C0F883040F4C77081E02B
:1027A00001C0880FCA95EAF70E94A91C183028F5C5
:1027B00081E09D2F977001C0880F9A95EAF70E94DB
:1027C000B41C802F0E94E91D1830F0F4D77081E00E
:1027D00001C0880FDA95EAF70AC080E28C0F8830D2
:1027E00098F4C77081E001C0880FCA95EAF7DF91BD
:1027F000CF911F910F910C94A91C802FDF91CF9145
:102800001F910F910C94E91DDF91CF911F910F91B2
:102810000895CF93DF93CFE6D0E060E0CE010E9431
:10282000C71E2196C11584E0D807B9F7DF91CF9173
:102830000895CF92DF92EF92FF920F931F93CF9361
:10284000DF93C0E0D0E08E010E5E1F4F6E0186E088
:10285000C80ED11CFE01E653FE4FE590F4906F2D9B
:10286000CE0187960E94C71E6E2DCE0188960E94CB
:10287000C71E2296CC15DD0569F70C171D0731F729
:10288000E80108341105F9F6DF91CF911F910F91FE
:10289000FF90EF90DF90CF9008950F931F93CF9309
:1028A000DF93C42FD0E0CC0FDD1F26E0629FC00D68
:1028B000D11D112432E1839FC00DD11D1124CE0101
:1028C00087960E94B91E082F10E0102F0027CE0116
:1028D00088960E94B91E9801282BC901DF91CF91DB
:1028E0001F910F910895462F843038F4733028F4E7
:1028F000633018F4672F0C944D1480E090E0089535
:102900000E943C092091D401211104C02091D501DD
:10291000222321F09093D1018093D0012091D60100
:10292000211104C02091D701222321F09093CE01E0
:102930008093CD01E091C901F091CA01309749F02F
:1029400082E08093D2010480F581E02D82ED91E058
:1029500009940895803F39F49091D50197FF35C0CF
:102960001092D50159C0813F29F49091D5011916D3
:10297000BCF32BC09091D401823F29F497FF25C06E
:102980001092D40149C0833F19F41916CCF31DC02D
:102990009091D601893F29F41916BCF41092D60102
:1029A0003BC08A3F19F497FF10C0F8CF8B3F39F432
:1029B0009091D70197FF09C01092D7012DC08C3F8D
:1029C00021F49091D7011916BCF39CE0980F953033
:1029D00080F421E030E0A90102C0440F551F9A9510
:1029E000E2F7CA0180959091D30189238093D301A6
:1029F00013C08D3F21F4809178018E7F0BC08E3FF4
:102A000021F4809178018D7F05C08F3F29F480915A
:102A100078018B7F809378018091D401811106C069
:102A20008091D501811102C01092CF018091D60111
:102A3000811106C08091D701811102C01092CC0192
:102A400008958091780180FD16C081FD16C082FD39
:102A500018C08091CC01882391F0883290F428E04E
:102A6000829FC001112468E270E00E94FB1E862F45
:102A7000672B29F007C082E0089584E0089581E083
:102A8000089588E008958091780180FD14C081FD4B
:102A900014C082FD16C08091CF01882381F084315B
:102AA00080F422E3829FC001112464E170E00E945F
:102AB000FB1E862F08958CE0089589E1089585E036
:102AC000089582E30895803F21F40E944315819583
:102AD00004C0813F29F40E9443158093D5010895D5
:102AE000823F21F40E944315819504C0833F29F45D
:102AF0000E9443158093D4010895893F19F40E94E0
:102B0000211505C08A3F31F40E94211581958093DB
:102B1000D60108958B3F21F40E942115819504C0B0
:102B20008C3F29F40E9421158093D70108959CE0E1
:102B3000980F953078F421E030E0A90102C0440FED
:102B4000551F9A95E2F7CA019091D301892B809382
:102B5000D30108958D3F21F48091780181600BC0ED
:102B60008E3F21F480917801826005C08F3F29F467
:102B7000809178018460809378010895EF92FF92AC
:102B80000F931F93CF93DF93E6ECF1E06BE071E0DE
:102B900089ECE82E81E0F82EC0E001E010E080E052
:102BA00090E050E09B01280F391FD9014C914F3F15
:102BB000D1F0242F22952F7030E0D90190962C91DE
:102BC00030E04F7002C0359527954A95E2F720FD19
:102BD00007C09801082E01C0220F0A94EAF702C02C
:102BE00020E030E0522B019683309105D9F68081A8
:102BF000851719F0508381E001C080E0C82B319621
:102C00006D5F7F4FEE16FF0651F6CC2349F081E051
:102C10008093E6010E943C099093E5018093E401D2
:102C20008091E6018823B1F08091E4019091E50163
:102C30000E942D09069770F08091C6018093DD01F6
:102C40008091C7018093DE018091C8018093DF01EC
:102C50001092E6018C2FDF91CF911F910F91FF9081
:102C6000EF900895CF93DF930E947314EC018238A4
:102C7000910559F1A0F48133910509F473C040F432
:102C80008932910509F467C08A9709F472C084C03B
:102C90008533910509F458C0C997B9F07DC0833ECA
:102CA000910571F138F4803E9105B1F0823E9105B5
:102CB00011F172C0863E9105B9F1873E9105C9F1C7
:102CC000843E910509F068C024C08091C40180FD54
:102CD0005DC081FD5BC060C08091C40180FD50C0BB
:102CE0008091C50180FF49C18091C40184FD43C129
:102CF000C3EED0E042C18091C40182FF3EC1F4CF57
:102D00008091C40182FD3FC08091C50180FD3EC01D
:102D1000EBCF8091C50181FF30C18091C40184FD5A
:102D20002AC1C7EED0E029C18091C40183FF25C12B
:102D3000F4CF8091C40183FD2CC08091C50181FF37
:102D4000ECCFC4EED0E019C18091C40185FF15C15C
:102D5000C9E2D0E012C18091C40185FF0EC1C5E374
:102D6000D0E00BC18091C40186FF07C1CAE2D0E068
:102D700004C18091C40186FF00C1C1E3D0E0FDC061
:102D8000C9E3D0E0FAC0C2EED0E0F7C0C0EED0E0B8
:102D9000F4C0C6EED0E0F1C0C11581E5D80708F057
:102DA00066C0C11520E5D207E0F0CE0174E096952B
:102DB00087957A95E1F783709C2F937021E030E03E
:102DC00002C0220F331F9A95E2F73C68382BCF7070
:102DD000C695C69540E2C49FE0011124C22BD32BB7
:102DE000CCC0C83ED10560F5C03ED10508F0C5C0D5
:102DF000C83AD105B0F4C53AD10540F0C55AD0E083
:102E0000CD5DDE4FC881D0E0D064B7C0C130D10500
:102E100009F4B3C008F4AFC0C430D10508F4ABC0A6
:102E2000ACC0CF3BD10508F0A6C0C85AD0E0CC0F4B
:102E3000DD1FCA5DDE4F0990D881C02DD4649DC0CE
:102E4000C11540E2D40758F4C11581E0D80708F055
:102E500094C0C03FD10508F48EC0D0658EC0C115A6
:102E600020E4D20708F487C0DF70D06A86C0C1159D
:102E700045E5D40708F042C0C11584E5D80728F01D
:102E8000DC2FCC27C46FD06A78C0C11523E5D207E8
:102E9000B0F0CE018370992721E030E002C0220F0C
:102EA000331F8A95E2F78C2F8695869540E2849FA2
:102EB000C0011124E901C82BD92BDA685EC0C11505
:102EC00042E5D40728F4DC2FCC27C16FD06A55C067
:102ED000CE018370992721E030E002C0220F331F1A
:102EE0008A95E2F78C2F8695869540E2849FC001F3
:102EF0001124E901C82BD92BDC683FC0C11589E535
:102F0000D807B8F4C11528E5D20728F0DC2FCC2764
:102F1000C06FD06A32C0C11546E5D40760F58C2F6A
:102F20000E947D128F71C82FD0E0DC2FCC27D06299
:102F300024C0C1158AE5D80780F48C2F8F700E94B9
:102F40007D1294E0D695C7959A95E1F7CF70D0E0C1
:102F5000DC2FCC27D069C82B10C0CE01905681152C
:102F6000904248F48D2F8F710E947D12DD27D06230
:102F70008F71D82B02C0C0E0D0E0CE01DF91CF919D
:102F800008950F931F9380911C0290911D02A091B0
:102F90001E02B0911F028C019D010670112722278D
:102FA0003327BC01CD01063011052105310511F48F
:102FB000686001C0677F1F910F910C949A0B1F935B
:102FC000CF93DF93CDB7DEB7AA970FB6F894DEBFE5
:102FD0000FBECDBFE4E1F2E08091F100819342E0C9
:102FE000EC31F407C9F780911502833009F462C00F
:102FF00030F4813071F0823009F49CC0B3C08A3063
:1030000009F488C08B3009F46DC0893009F0AAC07A
:1030100020C080911402813A09F0A4C08091E80098
:10302000877F8093E8008091180290911902892B84
:1030300021F460E280EF91E003C060E080E090E086
:1030400070E00E945B1E8091E8008B778093E8001F
:1030500089C080911402813209F084C080911802E5
:1030600090911902009719F0029709F07BC08091A6
:10307000E800877F8093E8008091E80082FD05C02A
:10308000809112028111F8CF6DC02091F3008091E0
:10309000F20090E0922B029729F48091F1008B7F4F
:1030A000813021F48091F1008093EF018091E8005C
:1030B0008B7754C080911402813A09F053C08091FB
:1030C000180290911902892B09F04CC08091E800F8
:1030D000877F8093E8008091E80080FFFCCF80919B
:1030E0000A0137C0809114028132E1F58091180203
:1030F00090911902892BB1F58091E800877F809328
:10310000E8000E94071E8091160280930A010E9427
:10311000360E28C080911402813221F58091E8009A
:10312000877F8093E8000E94071E8091170280939A
:10313000EE0118C080911402813AA1F48091E80058
:10314000877F8093E8008091E80080FFFCCF80912A
:10315000EE018093F1008091E8008E778093E80083
:103160000E94071E8091E80083FFDDC18091140258
:1031700090911502492F50E04A30510508F0D3C113
:10318000FA01ED57FF4F0C940F1F803821F0823861
:1031900009F0C9C108C080911002909111029923D1
:1031A00089F082600FC0809118028F70873008F01C
:1031B000BAC18093E9008091EB0085FB882780F9F4
:1031C0001092E9009091E800977F9093E800809337
:1031D000F1001092F10070C1282F2D7F09F0A3C1DA
:1031E000882319F0823061F09EC1809116028130EF
:1031F00009F099C1933009F080E0809311022EC04C
:103200008091160281112AC0809118028F702FEFD1
:10321000280F263008F087C18093E9002091EB0049
:1032200020FF1CC0933021F48091EB00806214C019
:103230009091EB0090619093EB0021E030E0A901C8
:1032400002C0440F551F8A95E2F74093EA0010929E
:10325000EA008091EB0088608093EB001092E90017
:103260008091E800877F8093E8000E94071E5BC181
:10327000811159C1109116021F778091E300807867
:10328000812B8093E3008091E800877F8093E800A2
:103290000E94071E8091E80080FFFCCF8091E30030
:1032A00080688093E300111102C082E001C083E0D6
:1032B0008093120238C18058823008F034C12091C6
:1032C0001602309117022C3D53E0350779F583E063
:1032D0008A838AE289834FB7F894DE01139620E04F
:1032E0003EE051E2E32FF0E050935700E49120FFDD
:1032F00003C0E295EF703F5FEF708E2F90E0EA30F1
:1033000010F0C79601C0C0968D939D932F5F243116
:1033100049F74FBF8091E800877F8093E8006AE219
:1033200070E0CE0101960E945B1EB4C0809118022D
:1033300090911902432F552743305105A9F068F4A5
:103340004130510509F4FEC04230510509F0EBC08F
:103350008BE590E0EAE2F3E04BC04132510529F100
:103360004232510589F1DFC0C901992781309105A9
:10337000A1F058F0029709F0D6C0E7E9F3E0E49134
:103380008E2F90E0E7E9F3E030C0EBECF3E0E4915E
:103390008E2F90E0EBECF3E028C0EDEBF3E0E4914E
:1033A0008E2F90E0EDEBF3E020C08330910508F024
:1033B000BAC0880F991FFC01E35EFE4F0190F081B7
:1033C000E02D89E090E014C08330910508F0ABC097
:1033D000FC01EE0FFF1FE95EFE4F0190F081E02D32
:1033E000DC01AC5EBE4F8C9190E0009709F49BC06D
:1033F0002091E800277F2093E80020911A02309165
:103400001B022817390708F4C90140E0009789F129
:1034100020911202222309F43DC02530D9F12091D8
:10342000E80023FD37C02091E80022FD2FC0209145
:10343000E80020FFEBCF4091F3002091F20030E054
:10344000342B009759F02830310540F444914093D3
:10345000F100319601972F5F3F4FF3CF41E02830C5
:10346000310509F040E02091E8002E772093E80034
:10347000CDCF4111CDCF0AC080911202882351F0E7
:10348000853041F08091E80083FD04C08091E80020
:1034900082FFF2CF8091E8008B778093E80043C0F1
:1034A000803809F040C08091E800877F8093E80071
:1034B000809113028093F1008091E8008E77D3CE43
:1034C000811131C0809116029091170299270297BD
:1034D00054F58091E800877F8093E80010911602F0
:1034E000109313020E94071E111106C08091E30081
:1034F00087FD02C081E001C084E08093120242E0B7
:1035000061EC81E00E94261E42E261EC84E00E94B0
:10351000261E42E261EC82E00E94261E42E260EC3E
:1035200083E00E94261E8091E80083FF10C08091F6
:10353000E800877F8093E8008091EB0080628093B1
:10354000EB0005C082E190E0E5E8F3E051CFAA96F8
:103550000FB6F894DEBF0FBECDBFDF91CF911F91A4
:1035600008951F920F920FB60F9211242F933F933D
:103570004F935F936F937F938F939F93AF93BF937B
:10358000CF93DF93EF93FF93C091E900CF708091C9
:10359000EC00D82FD17080FDD0E81092E900809126
:1035A000F000877F8093F00078940E94DF171092DC
:1035B000E9008091F00088608093F000CD2BCF70FF
:1035C000C093E900FF91EF91DF91CF91BF91AF914F
:1035D0009F918F917F916F915F914F913F912F912B
:1035E0000F900FBE0F901F901895E8EDF0E08081CE
:1035F0008E7F80831092E2001092DA001092E10038
:10360000A0EEB0E08C9181608C9380818F77808375
:1036100019BCA7EDB0E08C918E7F8C9380818F7E5A
:1036200080831092ED010895CF92DF92EF92FF9286
:103630000F931F93CF93DF93C8EDD0E088818F7EE7
:103640008883E7EDF0E080818160808384E082BF41
:1036500081E08093ED0188818E7F888302EE10E007
:10366000F80110821092DA0081EEC82ED12CF601FA
:10367000108288818F778883888180688883888199
:103680008F7D888319BC109212021092130210923F
:1036900011021092100290EEE92EF12CF7018081B8
:1036A0008B7F808388818160888342E060E080E056
:1036B0000E94261EF60180818E7F8083F801808122
:1036C00081608083808188608083F70180818E7F24
:1036D0008083888180618883DF91CF911F910F91D2
:1036E000FF90EF90DF90CF9008951F920F920FB64A
:1036F0000F9211242F933F934F935F936F937F9378
:103700008F939F93AF93BF93EF93FF938091E100CB
:1037100082FF09C08091E20082FF05C08091E10034
:103720008B7F8093E1008091DA0080FF2AC0809136
:10373000D80080FF26C08091DA008E7F8093DA0067
:103740008091D90080FF18C080E189BD82E189BDE8
:1037500009B400FEFDCF81E0809312028091ED015B
:1037600081110FC00E94F51A0E94141B8091E20083
:1037700084608093E20005C019BC1092120210927E
:10378000ED018091E10080FF17C08091E20080FF91
:1037900013C08091E2008E7F8093E2008091E2006E
:1037A00080618093E2008091D80080628093D8008D
:1037B00019BC85E0809312028091E10084FF2EC045
:1037C0008091E20084FF2AC080E189BD82E189BD49
:1037D00009B400FEFDCF8091D8008F7D8093D80082
:1037E0008091E1008F7E8093E1008091E2008F7EE6
:1037F0008093E2008091E20081608093E2008091FA
:103800001302882311F084E007C08091E30087FD54
:1038100002C081E001C083E0809312028091E10048
:1038200083FF27C08091E20083FF23C08091E100E5
:10383000877F8093E10082E080931202109213024E
:103840008091E1008E7F8093E1008091E2008E7F85
:103850008093E2008091E20080618093E20042E088
:1038600060E080E00E94261E8091F00088608093D6
:10387000F000FF91EF91BF91AF919F918F917F9158
:103880006F915F914F913F912F910F900FBE0F90CD
:103890001F9018952091E4003091E50095E6409145
:1038A000EC00842F817040FF23C08091E80080FDF0
:1038B0001DC080911202882399F0853099F0809183
:1038C000EB0085FD11C04091E4005091E500241704
:1038D000350729F3915011F09A01E1CF84E0089562
:1038E00082E0089583E0089581E0089580E00895DE
:1038F0004091E80042FFDDCF0895EF92FF920F93D1
:103900001F93CF93DF937C018B010E944A1C81118E
:1039100019C0E70101151105A1F08091E80085FDAE
:103920000AC08091E8008E778093E8000E944A1CCC
:10393000882381F307C089918093F1000150110918
:10394000E9CF80E0DF91CF911F910F91FF90EF9031
:103950000895882341F080959091BE01892380933A
:10396000BE010C94500A0895882339F09091BE014D
:10397000892B8093BE010C94500A0895882309F482
:1039800063C0823869F40E948A1381FF5DC069E3D5
:1039900088E591E00E9499090E94500A69E30EC0EF
:1039A000833891F40E948A1380FF4EC063E588E556
:1039B00091E00E9499090E94500A63E588E591E030
:1039C0000E9471090C94500A843869F40E948A1389
:1039D00082FF3AC067E488E591E00E9499090E945D
:1039E000500A67E4EBCF9CEF980F913A10F4682FE0
:1039F000E5CF90E2980F983088F4877021E030E0AE
:103A0000A90102C0440F551F8A95E2F7CA018095AB
:103A10009091BE0189238093BE01D4CF9BE5980F7E
:103A2000933020F480E090E00C94741398E5980FA4
:103A3000973120F480E090E00C945E13803F20F0FA
:103A40000E94AA140C9480140895CF93882309F43B
:103A5000BEC0C82F8238B1F40E948A1381FDB7C05E
:103A600069E388E591E00E9499090E94500A2FEFCE
:103A700081EE94E0215080409040E1F700C00000CA
:103A800069E317C08338E1F40E948A1380FD9FC068
:103A900063E588E591E00E9499090E94500A2FEFA2
:103AA00081EE94E0215080409040E1F700C000009A
:103AB00063E588E591E00E947109CF910C94500A6A
:103AC0008438B1F40E948A1382FD81C067E488E5DE
:103AD00091E00E9499090E94500A2FEF81EE94E034
:103AE000215080409040E1F700C0000067E4E1CF42
:103AF0008CEF8C0F813AC0F580910A018823E1F0A8
:103B00008091C40187FF18C0EC2FE695E695E695F5
:103B1000F0E0E85AFE4F8281282F30E04C2F4770AA
:103B200081E090E002C0880F991F4A95E2F7822356
:103B30009323892B61F412C0EAE5F1E080E691E07D
:103B40002191C21721F08E179F07D1F707C06C2F64
:103B500088E591E00E9471090E94500A6C2F88E567
:103B600091E00E949909A9CF80E28C0F883068F417
:103B7000C77081E090E001C0880FCA95EAF7909184
:103B8000BE01892B8093BE0198CFEBE5EC0FE330AB
:103B900040F4F0E0ED5DFE4F808190E0CF910C9419
:103BA0007413E8E5EC0FE73150F4F0E0EE0FFF1F7F
:103BB000EA5DFE4F80819181CF910C945E13C03FEE
:103BC00030F08C2F0E946315CF910C948014CF910C
:103BD00008951F93CF93DF93182F893319F0C0E016
:103BE000D0E002C0C0E5D0E0812F0E94251D2097C3
:103BF00041F08FE99FE00197F1F700C000002197A5
:103C0000F6CF812FDF91CF911F910C94BE1C809134
:103C1000140287FF11C08091E80082FD05C08091E9
:103C200012028111F8CF11C08091E8008B770BC090
:103C300080911202882349F08091E80080FFF8CF3C
:103C40008091E8008E778093E8000895982F973050
:103C500068F59093E900981739F07091EC00209185
:103C6000ED005091F00003C0242F762F50E021FD8D
:103C700002C09F5FECCF3091EB003E7F3093EB00B2
:103C80003091ED003D7F3093ED003091EB003160DD
:103C90003093EB007093EC002093ED005093F00014
:103CA0002091EE0027FDE5CF80E008958F7080938E
:103CB000E90081E0089520911A0230911B02261735
:103CC000370748F06115710539F42091E8002E7727
:103CD0002093E80001C0B901FC0120E061157105E5
:103CE00079F1809112028823F1F18530F1F1809110
:103CF000E80083FD3CC08091E80082FD2EC08091E9
:103D0000E80080FFEBCF2091F3008091F20090E07B
:103D1000922B6115710551F08830910538F421918D
:103D20002093F100615071090196F3CF21E00897CB
:103D300009F020E08091E8008E778093E800CECFF4
:103D40002111CFCF0AC080911202882361F0853003
:103D500061F08091E80083FD0AC08091E80082FF55
:103D6000F2CF80E0089582E0089583E0089581E035
:103D70000895F999FECF92BD81BDF89A992780B533
:103D80000895A8E1B0E042E050E00C94ED1E262F2B
:103D9000F999FECF92BD81BDF89A019700B4021641
:103DA00039F01FBA20BD0FB6F894FA9AF99A0FBEEF
:103DB00008950396272F0E94C81E0E94C71E252F14
:103DC0000E94C81E242F0C94C81E0196272F0E9403
:103DD000C81E0C94C71EDC01CB01FC01F999FECF73
:103DE00006C0F2BDE1BDF89A319600B40D92415083
:103DF0005040B8F7089597FB072E16F4009407D0AB
:103E000077FD09D00E941C1F07FC05D03EF4909559
:103E100081959F4F0895709561957F4F0895EE0F9E
:103E2000FF1F0590F491E02D0994692796276927D3
:103E30007827872778270895AA1BBB1B51E107C065
:103E4000AA1FBB1FA617B70710F0A61BB70B881F2A
:103E5000991F5A95A9F780959095BC01CD010895B9
:043E6000F894FFCF04
:103E64005F08830864084F0E4B0E01F4F5F6F73132
